:100000008A150A160028FF3FFF00030E8301EE0049
:100010000A08ED008A017008A2007108A100040816
:10002000A30083168C1E802883128C1E80281A0839
:100030000317B2000313981C302818121816500822
:10004000013EF00000300318013E5107F100700836
:10005000D0007108D1001A080317B200B20180283D
:100060000313181D42285008013EF0000030031809
:10007000013E5107F1007008D0007108D10003174C
:10008000B201802803131A080317B20032080D3A90
:1000900003195728803003135E06F0008030700289
:1000A000031D542820305D020318572868280313C5
:1000B0008316E41683125D082A3E840080015D08E1
:1000C000DB005E08DC00DD01DE010317B2018028E1
:1000D00003135D082A3E84000317320880000313CF
:1000E0005D08DB005E08DC005D08013EF0000030CA
:1000F0000318013E5E07F1007008DD007108DE00A4
:100100008B1EA6280B1DA628831203130B113C304F
:1001100081005F08013EF00000300318013E6007D7
:10012000F1007008DF007108E00080306006F00028
:1001300080307002031D9E2864305F02031CA628D5
:10014000831664158312DF01E001F727831203137E
:100150002208F0002108F100230884006D088A00BD
:100160006E0E8300FF0E7F0E090083120313F2014F
:10017000F30180307306F00080307002031DC22846
:10018000083072020318DB2803138711803003172D
:100190003105F1007108803A031DD12803130716B9
:1001A000D3280313071287150317B10D3110F20A74
:1001B0000319F30AB9280800831203137008F10029
:1001C000F0010830FC007108F40C0318EB28FC0B5C
:1001D000E428F10100340310F028F40C0318F107AF
:1001E000F10CF00CFC0BED280800FB14FB1FFF28A2
:1001F000FF30F300F200F100F000FA0DF20CFF30D6
:100200000800FA1FF213003008007B15FB1F0F29AE
:100210000130F300F201F101F001FA0DF20CFF30B0
:100220000800F201F101F001F801F30100300800CB
:100230008316031363088A00620882000800831291
:1002400003138714071003173008B100B520831279
:10025000031307140800A0017208031D4029710848
:10026000F2007008F100F001A0157208031D40298A
:100270007108F200F101A0112016720803194E292D
:100280002008F302031D031C52290310F21B5629F8
:10029000F00DF10DF20DF30B462952290130FC004F
:1002A000112159290230FC00052159290430FC0094
:1002B000012108007C189029FC1861297C19AF29BC
:1002C0005A29A0017208031D81297108F2007008E3
:1002D000F1007808F000F801A0157208031D8129CB
:1002E0007108F2007008F100F001A01120167208E8
:1002F000031D81297108F200F101A015720803198C
:10030000A3292008F302031D031CA7290310F21BD5
:100310009029F80DF00DF10DF20DF30B8729A729A7
:100320007B1B701CAB29F81FAB29F00A0319F10ADB
:100330000319F20A031DAB29F20CF10CF00CF30ABD
:100340000319AF29AB290130FC001121B229023079
:10035000FC000521B2290430FC000121B22908303B
:10036000FC00F52000000800831603139818BA2932
:100370000000B429831203172B0803139900080007
:10038000831203172B08F2007208F000F20A7008BB
:10039000840000080319CD29C4292B087202F0003B
:1003A0000130F002F101031CF10308000630840063
:1003B0000008000883120313F00070137008800017
:1003C00008000000000008002030831203172B02F1
:1003D000031CEF292B087F3C031CEF29F0292D2A51
:1003E0000530F0002B08F400DC20A0307002031769
:1003F000AC000030031C013E7102AD000530AE00C0
:100400000030AF008030F00080302F067002031DF6
:100410000B2A2E08003C03182B2A2C08233EF00040
:1004200014300318013E2D07F100700883160313E2
:10043000E2007108E30018218A110A1283120317DF
:10044000B0001F210317AC0A0319AD0A0130AE0238
:10045000031CAF03022AB0011F21080083120313FB
:100460008710071003172B08B100B5202130831225
:100470000313FC007630FD00FD0B3C2AFC0B3C2AEC
:1004800000000714080006308400000800088312EA
:100490000313F000F01370088000080083120317A4
:1004A000A701A8018030A9000030AA0029082A0469
:1004B00003197C2AE121E121831603138617E12128
:1004C000E121061783126110061B6A2A611C692A42
:1004D0006A2A642A861F712A03172908A7042A0892
:1004E000A804E121E121D621831606138312031704
:1004F000AA0CA90CAA13562A831603138617E12106
:10050000E121831203172508260403198A2A4322AE
:100510008316861383160313E121E1210617831244
:100520006110061B972A611C962A972A912AE121BD
:10053000E121D62183160613E121E121432283160E
:100540008613831203172708F0000800831203178D
:100550002608003C0318C52A093026020318C52ABC
:100560002603F0000730F00540307004AB002E2267
:1005700003172508F0000630F400DC207F30F0057A
:10058000803070040317AB002E220800831203137F
:10059000F801F9011030FC00710DF80DF90D740827
:1005A000F8027508031C750FF9020318DE2A740897
:1005B000F80775080318750FF9070310F00DF10D12
:1005C000FC0BCC2A08008312031372087606A000E5
:1005D000F801F90173087702031C062B7708FD0068
:1005E0007308F7007D08F3007608FD007208F60036
:1005F0007D08F2007508FD007108F5007D08F10026
:100600007408FD007008F4007D08F00077080319F5
:100610007F2B7208FA00F217F61777087302F700BB
:100620000319392B08307702031C2F2BF7007408AD
:10063000F9007508F4007608F500F6010830770235
:10064000031C2F2BF7007408F9007508F400F5015E
:1006500008307702031C2F2B7A08F2007F2B7708D3
:100660000319392B0310F60CF50CF40CF90CF70BED
:10067000322BA01F462BF909F409F509F609F90AEE
:100680000319F40A0319F50A0319F60A7908F80799
:1006900074080318740FF00775080318750FF10735
:1006A00076080318760FF207A01B5F2B031C6F2B35
:1006B000F20CF10CF00CF80CF30F6F2B7B2B0318E2
:1006C000732BF809F009F109F209F80A0319F00A85
:1006D0000319F10A0319F20A8030FA06772B013068
:1006E000FC005A21812B0230FC005A21812B04305E
:1006F000FC002B21812B0830FC00F520812B0030E1
:10070000FC0000000800831203172508393C031C75
:10071000902B30302502031C902B0130F000912BE0
:10072000F001080083120313FB01FA01F901803084
:10073000F800F10CF00C031CA62B7408F9077508DF
:100740000318750FFA070318FB0A0310F01FAE2BEE
:100750007408FA0775080318750FFB07FB0CFA0CF1
:10076000F90CF80C031C992B7B08F3007A08F200B3
:100770007908F1007808F0000800831203172508B3
:10078000AB00C0217008A700A60126082507840039
:100790000008A80083160313641BD42B83120317CD
:1007A0002808AB00B421D92B831203172808AB000B
:1007B000E42183120317A60A80302606F000803059
:1007C00027067002031CC52B08007B14FB1FF02BAF
:1007D000F201FA1FFF30F200F100F000FA0DF20C06
:1007E000FF300800FB15FF3008008316031386173F
:1007F000E121E1210617E121E1214322831686133D
:10080000E121E121D621831606130800013083126D
:100810000317A8000030A9008030A600A701260811
:10082000270403193F2CE121E121E121E121D62117
:1008300083160613E121E1218312031726082505FB
:10084000F00000302705F1007008710403192C2C0A
:100850008316031386172F2C432283168613E12158
:10086000E121061783126110061B3A2C611C392CFA
:100870003A2C342C0317A70CA60CA7130F2CA80195
:10088000A901E121E121D62183160613E121E1210D
:100890008617E121E121E121E12106178312611090
:1008A000061B562C611C552C562C502C0317A801E6
:1008B000A901E121E121861F5E2C2814E121E1211B
:1008C000E121E121E121E121E121E121E121E12118
:1008D000E121E121E121E121E121E121D62183167C
:1008E0000613432283168613831203172808F00089
:1008F000080083120313F8010830FC00700DF80D96
:100900007408F8020318862CF8070310F00DFC0B8E
:100910007E2C0800432283168613E121E12106176D
:1009200083126110061B982C611C972C982C922C1A
:10093000E121E121E121E121E121E121E121E121A7
:1009400083168617E121E1210800F523D0308312B8
:100950000317A5000624700883160313E100831211
:100960000317A5010624700883160313E1008030E5
:1009700083120317A5000624700883160313E100F1
:10098000831254080317A500062470088316031366
:10099000E100831253080317A5000624700883168C
:1009A0000313E100831258080317A50006247008FA
:1009B00083160313E100831257080317A5000624CA
:1009C000700883160313E100831256080317A5006D
:1009D0000624700883160313E100831252080317DC
:1009E000A5000624700883160313E1008A24F5236A
:1009F0002130FC007630FD00FD0BFC2CFC0BFC2CA8
:100A00000000D03083120317A50006247008831657
:100A10000313E10083120317A5010624700883164F
:100A20000313E10083120317A5010624700883163F
:100A30000313E1008A24080083120317A0011E0893
:100A4000840000089F001F08003A0319322D1F0878
:100A5000AB00B4210317A00A20081E078400000879
:100A60009F00232D080083120317A00103302002EA
:100A70000318412D20081F07840020308000A00AA1
:100A8000362D20081F0784008001A00320081F07BF
:100A9000A1000A30F4001E08F00079247808F00064
:100AA0003030F007031721088400700880000A30F6
:100AB000F4001E08F0007924700803179E007008E7
:100AC000003A031D642D662DA003462D08008312F5
:100AD0000313FA017308031D7A147708031DFA142F
:100AE0007A080319B32D033A03197E2D7A187B2D4A
:100AF000F61FB12DAF2DF21FAF2DB12D7208803929
:100B0000FA00F21376088039F6137A0603198C2D51
:100B10007A080319AF2DB12D770873020319932DAD
:100B2000031CA72DAB2D7608720203199A2D031C06
:100B3000A72DAB2D750871020319A12D031CA72D3C
:100B4000AB2D740870020319B32D0318AB2DFA08EE
:100B50000319B12DAF2DFA080319AF2DB12D0314D0
:100B600008000310080003140315080008000130F2
:100B700083120317A5000130A600A622213083129C
:100B80000313FC007630FD00FD0BC42DFC0BC42DBF
:100B9000000003179E019F0180301F06F000803087
:100BA000033A7002031DD62D00301E020318E92DF2
:100BB000B0011F210430FC003D30FD00FD0BDE2D97
:100BC000FC0BDE2D0000000003179E0A03199F0A8C
:100BD000CC2D0800F523A03083120317A5000624AE
:100BE000700883160313E100831203171F08F00037
:100BF000F1017008A5000624700883160313E100B4
:100C0000FF30831203171E05A50006247008831603
:100C10000313E100831203172008A50006247008BF
:100C200083160313E1008A241130FC003A30FD00E2
:100C3000FD0B182EFC0B182E000008000D3083123F
:100C40000317AB00B4210A300317AB00B42108002E
:100C5000831203171F0883160313E200831203177E
:100C6000200883160313E30018218A110A12F000EA
:100C700070080319562E831203171F0883160313D7
:100C8000E20083120317200883160313E3001821E0
:100C90008A110A12F000831203171E0884007008DC
:100CA00080009E0A9F0A0319A00A282E83120317A8
:100CB0001E08840080010800831203137008F800E6
:100CC0007108F000F101F201F301FB01FC01963023
:100CD000F300FA01F01F722EF809F009F80A03195F
:100CE000F00AFA177008F1007808F000F801F20134
:100CF0002B210800831203179F011E08093C0318CB
:100D00009E2E0A30F4001E08F000792470080317A4
:100D10009F0070089F009F0D1F109F0D1F109F0DBB
:100D20001F109F0D1F100A30F4001E08F0007924D8
:100D30007808F000700803179F04A02E1E089F007B
:100D40001F08F000080083120313FB017308031946
:100D5000E02E7208FA00F2178E30F302F31FE32E32
:100D6000F309F30A08307302031CC62EF300F10DD9
:100D70007208F100F20108307302031CC62EF30062
:100D8000F10DF1017308031D0310CE2E7308031932
:100D9000CE2E0310F20CF10CF30BC92E7B1B711C31
:100DA000D82E031CD82EF10A0319F20AF21BEF2EDB
:100DB000FA1FF22EF209F109F10A0319F20AF22ED2
:100DC000F201F101F22E7B14FB1FF52EF201FA1F46
:100DD000F52EFF30F200F100FA0DF20CF52E013085
:100DE000FC00F72E0030FC00F72EFF30FC00FC0862
:100DF0000319FB2EE5237108F0007208F1000800CA
:100E000083120313FB01FC01FA01730803193F2F3E
:100E1000F2178E30F302F31B102F0319102F422FFD
:100E2000F309F30A08307302031C252FF300F10DB8
:100E30007208F100F20108307302031C252FF10D36
:100E4000F1017308031D03102D2F730803192D2FB3
:100E50000310F20CF10CF30B282F7B1B711C372FA6
:100E6000031C372FF10A0319F20AF21B4E2FFA1F47
:100E7000512FF209F109F10A0319F20A512FF20177
:100E8000F101512F7B14FB1F542FF201FA1F542F35
:100E9000FF30F200F100FA0DF20C542F0130FC008B
:100EA000562F0030FC00562FFF30FC00FC080319C1
:100EB0005A2FE5237108F0007208F1000800831230
:100EC00003171E08840000089F00A0010030A00046
:100ED00000302006031D6E2F20301F060319792FC6
:100EE00000302006031D762F09301F060319792FC5
:100EF0007B2F9E0A5F2FA101A201A301A401003054
:100F00002006031D852F2D301F06031D8C2FA30ADD
:100F10000319A40A9E0A952F00302006031D922F64
:100F20002B301F06031D952F9E0A1E088400000803
:100F30009F00A0010030A0001F08A50083237008B7
:100F40000319BE2F2108F0002208F1000A30F40036
:100F50000030F5009223303003171F02F2000030FA
:100F6000031C013E2002F30072087007A100710803
:100F70000318013E7307A2009E0A952F230824043C
:100F80000319CB2F2108003CF0002208031C013E6E
:100F9000F101F102CF2F2108F0002208F100080032
:100FA000831203138030F606E3220800831203172E
:100FB0002008A5001E08A600A622831203172208F7
:100FC000AB00E421080018218A110A128000840A6B
:100FD000E20A0319E30AF003031DE32F080081303E
:100FE000831203139F008E3083169F000800831224
:100FF000031361140800FF3FFF3FFF3FFF3FFF3F28
:10100000831203171E0883160313E20083120317CB
:101010001F0883160313E3008A1118218A150A1288
:10102000F000700803192F28831203171E08831677
:101030000313E200831203171F0883160313E30050
:101040008A1118218A150A1283120317AB008A111C
:10105000B4218A1503179E0A03199F0A0028080065
:1010600083120317A1010530210203183E2821082D
:101070002007840020308000A10A3328210820079F
:1010800084008001A10321082007A2000A30F40097
:10109000F5011E08F0001F08F1008A11C6228A150A
:1010A0007808F0007908F1003030F00703172208C3
:1010B0008400700880000A30F400F5011E08F0007A
:1010C0001F08F1008A11C6228A15700803179E00B6
:1010D00071089F0000307106031D702800307006F3
:1010E000031D73287528A1034328080083120313E6
:1010F0007408003A031D91287508003A031D9128D1
:101100007608003A031D91287708003A031D9128BC
:10111000FF30F000FF30F1007F30F200FF30F300CD
:10112000342983120313770803192029730803193C
:101130002529720876068039FA00F217F617A00101
:101140007208F8007108FC007008FD007408FD02C8
:101150007508031C750FFC027608031C760FF80255
:10116000F801FC01FD01031CBC280310F20CF10C7A
:10117000F00CF80C0130A0007708F302031CC6281D
:101180007E302007F30703182A29CB287E3020075A
:10119000F307031C2F291830FA07FD0DFC0DF80D7D
:1011A000F00DF10DF20DA00D7408F0027508031C8E
:1011B000750FF1027608031C760FF202760DA0047B
:1011C000201CE4287D14EF287408F0077508031824
:1011D000750FF10776080318760AF2077D10FA03F7
:1011E0001F307A05031DCD287B1B7D1C162903109B
:1011F000F00DF10DF20DA00D7408F0027508031C3E
:10120000750FF1027608031C760FF202760D2004AA
:101210000139FD070318FC0A0319F80A031D1629F2
:10122000F80CFC0CFD0CF30A03192A29FA1FF81319
:101230007808F2007C08F1007D08F00000303329C6
:1012400001308A11F2238A15332902308A111121C3
:101250008A15332904308A11F5208A15332908307C
:101260008A1105218A1500000800831603136413F0
:10127000831203172008A5008A11BD238A150030A8
:101280001F06031D452901301E06031D52290A3081
:10129000AB008A11B4218A150D300317AB008A11F7
:1012A000B4218A15031383166417080083120313ED
:1012B000FB017308031D77080319AD297208760630
:1012C000FA007708F3077E30031C6A29F30203183B
:1012D000B2296D29F302031CB7297208F8007108BE
:1012E000FC007008FD00F817F6170310F201F10179
:1012F000F0011830A0007D1C87297408F0077508DC
:101300000318750FF10776080318760FF207F20C31
:10131000F10CF00CF80CFC0CFD0C0310A00B7B295D
:10132000F21B9729F80DF00DF10DF20DF3037B1B65
:10133000701CA929F81FA929F00A0319F10A031939
:10134000F20A031DA929F20CF10CF00CF30A03199F
:10135000B229FA1FF2130030BB2901308A11112182
:101360008A15BB2902308A11F5208A15BB29043061
:101370008A1105218A15000008008A11F5238A15B3
:10138000D03083120317A5008A1106248A1570082D
:1013900083160313E10083120317A5018A110624A3
:1013A0008A15700883160313E1008A118A248A15AE
:1013B0008A11F5238A151130FC003A30FD00FD0B2F
:1013C000DF29FC0BDF290000D13083120317A500B1
:1013D0008A1106248A15700883160313E10004306D
:1013E000FC003D30FD00FD0BF329FC0BF329000050
:1013F0000000013083120317A5000030A6008A11F7
:101400004E228A151E088400700880000130A50055
:101410000030A6008A114E228A151F088400700829
:1014200080000130A5000030A6008A114E228A15E6
:1014300020088400700880000130A5000030A6005C
:101440008A114E228A15210884007008800001301C
:10145000A5000030A6008A114E228A1522088400B9
:10146000700880000130A5000030A6008A114E22CD
:101470008A152308840070088000A501A6018A113E
:101480004E228A1524088400700880008A118A245C
:101490008A15080083160313641783126F08031755
:1014A0009E000630F0000030F10083160313670839
:1014B000F400F5018A1192238A157008763E03170D
:1014C0009F0016300318013E7107A0008A112826DC
:1014D0008A1503136F080317A5008A11BD238A1507
:1014E0009E019F0103136F080317A00035216417A5
:1014F00083120317A5010230A6008A11A6228A15BD
:101500000230831203179E0000309F000530A000B8
:101510000030A1002030A2008A11D6278A1502309F
:10152000831203179E0000309F000630A000003099
:10153000A1000A30F400831603136808F0008A1132
:1015400079248A15303070070317A2008A11D62734
:101550008A150230831203179E0000309F00073067
:10156000A0000030A1000A30F400831603136808BD
:10157000F0008A1179248A157808F000303070075D
:101580000317A2008A11D6278A1502308312031787
:101590009E0000309F000830A0000030A1002F30D6
:1015A000A2008A11D6278A150230831203179E00E3
:1015B00000309F000930A0000030A1000A30F40084
:1015C000831603136908F0008A1179248A153030D4
:1015D00070070317A2008A11D6278A1502308312DA
:1015E00003179E0000309F000A30A0000030A100C9
:1015F0000A30F400831603136908F0008A11792475
:101600008A157808F000303070070317A2008A119D
:10161000D6278A150230831203179E0000309F00E0
:101620000B30A0000030A1002F30A2008A11D62775
:101630008A150230831203179E0000309F000C3081
:10164000A0000030A1003230A2008A11D6278A15EE
:101650000230831203179E0000309F000D30A0005F
:101660000030A1003030A2008A11D6278A1502303E
:10167000831203179E0000309F000E30A000003040
:10168000A1000A30F400831603136A08F0008A11DF
:1016900079248A15303070070317A2008A11D627E3
:1016A0008A150230831203179E0000309F000F300E
:1016B000A0000030A1000A30F400831603136A086A
:1016C000F0008A1179248A157808F000303070070C
:1016D0000317A2008A11D6278A15831603136413F1
:1016E0006808C0006808831203179E00C9309F0075
:1016F0008A1133258A15C9309E008A111C258A1546
:101700002F30AB008A11B4218A1583166908C100F5
:101710006908831203179E00C9309F008A11332580
:101720008A15C9309E008A111C258A152F30AB00FE
:101730008A11B4218A1583166A08C2006A088312C6
:1017400003179E00C9309F008A1133258A15C930BE
:101750009E008A111C258A15831603136708C3008F
:101760003B3083120317AB008A11B4218A1508009D
:1017700083160313641783120317A5010130A60013
:101780008A11A6228A15831203136F0803179E007D
:10179000CE309F001730A0008A1128268A15031327
:1017A0006F080317A5008A11BD238A159E019F01AA
:1017B00003136F080317A0003521013083120317AC
:1017C000A5000130A6008A11A6228A1501308312D5
:1017D00003179E0000309F000730A0000030A100DA
:1017E0000A30F400831603136908F0008A11792483
:1017F0008A15303070070317A2008A11D6278A1580
:101800000130831203179E0000309F000830A000B3
:101810000030A1000A30F400831603136908F000B9
:101820008A1179248A157808F00030307007031780
:10183000A2008A11D6278A150130831203179E0051
:1018400000309F000930A0000030A1003A30A20013
:101850008A11D6278A150130831203179E000030A3
:101860009F000A30A0000030A1000A30F400831667
:1018700003136808F0008A1179248A153030700744
:101880000317A2008A11D6278A1501308312031785
:101890009E0000309F000B30A0000030A1000A30F5
:1018A000F400831603136808F0008A1179248A155E
:1018B0007808F000303070070317A2008A11D6278D
:1018C0008A150130831203179E0000309F000C30F0
:1018D000A0000030A1003A30A2008A11D6278A1554
:1018E0000130831203179E0000309F000D30A000CE
:1018F0000030A1000A30F400831603136708F000DB
:101900008A1179248A15303070070317A2008A11D2
:10191000D6278A150130831203179E0000309F00DE
:101920000E30A0000030A1000A30F400831603132B
:101930006708F0008A1179248A157808F0003030A1
:1019400070070317A2008A11D6278A150130831267
:1019500003179E0000309F000F30A0000030A10050
:101960002030A2008A11D6278A1583160313641328
:101970006908C4006908831203179E0024309F0081
:101980008A1133258A1524309E008A111C258A1558
:101990003A30AB008A11B4218A1583166808C50055
:1019A0006808831203179E0024309F008A11332594
:1019B0008A1524309E008A111C258A153A30AB0006
:1019C0008A11B4218A1583166708C6006708831236
:1019D00003179E0024309F008A1133258A15243076
:1019E0009E008A111C258A153B30AB008A11B42158
:1019F0008A150800831603136B08EF006C08003C7F
:101A0000031C072D0730ED000030EE00262D6C087A
:101A1000163C0318122D1730831203179000003064
:101A200091001C2D831603136C08013E83120317CB
:101A3000900091010318910A100883160313ED001A
:101A400083120317110883160313EE006D08831227
:101A500003179800831603136E0883120317990067
:101A600092019301F401F501F601F70183160313C6
:101A70006708F0006808F1006908F2006A08F300DE
:101A80008A1167258A15013003180030F0007008AC
:101A90000319582D83166B0884002D308000EB0A43
:101AA0000030E7060030E8068030E9060030EA063C
:101AB00083166708F4006808F5006908F6006A08EC
:101AC000F700F001F101F201F3018A1167258A158F
:101AD000013003180030F00070080319AD2D031316
:101AE0000030F4000030F5000030F6007F30F700E1
:101AF00083166708F0006808F1006908F2006A08B8
:101B0000F3008A1167258A15013003180030F000B0
:101B100070080319AD2D83166708F0006808F100FE
:101B20006908F2006A08F3000030F4000030F500A4
:101B30002030F6008230F700562170088316E70047
:101B40007108E8007208E9007308EA0001308312A6
:101B500003179202031C93036F2D0030F400003032
:101B6000F5002030F6008230F70083160313670873
:101B7000F0006808F1006908F2006A08F3008A11B1
:101B800067258A150130031C0030F0007008031926
:101B9000EA2D0030F4000030F5002030F6008230ED
:101BA000F70083166708F0006808F1006908F20082
:101BB0006A08F300762070088316E7007108E800D1
:101BC0007208E9007308EA0083120317920A0319E6
:101BD000930AAD2D03171208980713080318013E46
:101BE0009907013094000030950000309A000030D1
:101BF0009B0000309C007F309D0080301506F00077
:101C0000803019067002031D072E180814020318ED
:101C1000272E0030F4000030F5002030F60082302E
:101C2000F7001A08F0001B08F1001C08F2001D085C
:101C3000F3007620700803179A0071089B00720861
:101C40009C0073089D00940A0319950AFD2D00302D
:101C5000F4000030F5000030F6008030F7001A087C
:101C6000F0001B08F1001C08F2001D08F3007620AC
:101C700083166708F4006808F5006908F6006A082A
:101C8000F7008A11E3228A1570088316E7007108AD
:101C9000E8007208E9007308EA000030F400003040
:101CA000F5002030F6008230F7008A1167258A158A
:101CB0000130031C0030F000700803196D2E003055
:101CC0008316E7000030E8000030E9007F30EA00CA
:101CD00083120317920A0319930A0317803013061D
:101CE000F00080307002031D772E003012020318BE
:101CF000B62E831603136B08840030308000EB0A85
:101D00006B0884002E308000EB0A803083120317AA
:101D10001906F00080307002031D902E003018026A
:101D20000318982E18089202031C930319089302B3
:101D3000FF309400FF30950080301306F0008030B3
:101D400015067002031DA62E140812020318B62EE3
:101D5000831603136B08840030308000EB0A0130D7
:101D6000831203179402031C95039C2E9401950182
:101D700080301506F000803019067002031DC22E57
:101D8000180814020318382F831603136708F0008D
:101D90006808F1006908F2006A08F3008A11A326B6
:101DA0008A15700803179600710897003030F00705
:101DB000831603136B08840070088000EB0A8312FB
:101DC000031715081306031DE72E12081406031D3A
:101DD000F02E831603136B0884002E308000EB0A6C
:101DE000831203171608F0001708F1008A115C2609
:101DF0008A15700803179A0071089B0072089C00EE
:101E000073089D007008F4007108F5007208F60070
:101E10007308F700831603136708F0006808F100E1
:101E20006908F2006A08F3008A11D0278A15700841
:101E30008316E7007108E8007208E9007308EA00F9
:101E40000030F4000030F5002030F6008230F7005A
:101E5000562170088316E7007108E8007208E9004F
:101E60007308EA0083120317940A0319950AB82E1F
:101E7000831603136B08840080016F08F0000800CC
:101E8000831203137008F8007108F000F101F201E9
:101E9000F301FB01FC019630F300FA017008F10038
:101EA0007808F000F801F2018A112B218A15080048
:101EB000831603136708073C0318612FF001F10133
:101EC000862FC73083129F0583166708F000F00D38
:101ED0007010F00D7010F00D7010700883129F04D8
:101EE0000A30FC00BC30FD00FD0B742FFC0B742F7E
:101EF00000001F1500001F1D7E2F7B2F1E08F10004
:101F0000F00183161E08F0070318F10A08008A1171
:101F1000F5238A15A03083120317A5008A11062421
:101F20008A15700883160313E1006808F000F101B8
:101F3000700883120317A5008A1106248A157008F9
:101F400083160313E100FF30670583120317A50012
:101F50008A1106248A15700883160313E1008A117A
:101F60008A248A158A11F5238A150430FC003D3035
:101F7000FD00FD0BB92FFC0BB92F00000000A130B4
:101F800083120317A5008A1106248A157008831688
:101F90000313E10083120317A501A6018A114E2243
:101FA0008A15700883160313E9008A118A248A159A
:101FB0006908F000080083120313D5015930D400DA
:101FC0001330D3000430D7000630D6000430D800D8
:101FD0001430D2008A11A5248A1508008316031331
:101FE0000617861783126110061BFA2F611CF92F42
:101FF000FA2FF42F0800FF3FFF3FFF3FFF3FFF3F57
:1020000083160313670884000008EE007F306E0516
:10201000F2007208F000F00CF013F00CF013F00C6A
:10202000F013F00CF0130A30F4000A12DC200A1648
:102030000F3083166E05F1007108F0076708840001
:1020400070088000680884000008EE00F0306E051B
:10205000F2007208F000F00CF013F00CF013F00C2A
:10206000F013F00CF0130A30F4000A12DC200A1608
:102070000F3083166E05F1007108F00768088400C0
:1020800070088000690884000008EE0030306E059A
:10209000F2007208F000F00CF013F00CF013F00CEA
:1020A000F013F00CF0130A30F4000A12DC200A16C8
:1020B0000F3083166E05F1007108F007690884007F
:1020C000700880006A08840007300005F0006A0884
:1020D0008400700880006B0884000008EE00F03077
:1020E0006E05F2007208F000F00CF013F00CF01323
:1020F000F00CF013F00CF0130A30F4000A12DC209C
:102100000A160F3083166E05F1007108F0076B0890
:102110008400700880006C0884000008EE00103015
:102120006E05F2007208F000F00CF013F00CF013E2
:10213000F00CF013F00CF0130A30F4000A12DC205B
:102140000A160F3083166E05F1007108F0076C084F
:102150008400700880006D0884000008EE00F030F4
:102160006E05F2007208F000F00CF013F00CF013A2
:10217000F00CF013F00CF0130A30F4000A12DC201B
:102180000A160F3083166E05F1007108F0076D080E
:10219000840070088000080083120317A5018316CD
:1021A0000313670883120317A6000A12A6220A1651
:1021B000213083120313FC007630FD00FD0BDE2876
:1021C000FC0BDE280000013083166702F0000030AF
:1021D000031C013E6802F1006030F4000030F5009D
:1021E0000A1292230A16603070078316E9007108FC
:1021F0000318013EEA007008E7007108E80080302B
:102200006806F00080306A067002031D092969081B
:1022100067020318202983120317B0010A121F2135
:102220000A160430FC003D30FD00FD0B1529FC0BA7
:102230001529000000008316E70A0319E80AFF28A1
:1022400083120317A501831603136708831203176C
:10225000A6000A12A6220A16073083120313FC00F6
:102260007D30FD00FD0B3229FC0B3229080083165E
:1022700003136708F0006808F1000A125C260A16CA
:102280000030F4000030F5004030F6008530F700F3
:102290008A150A1256218A110A160030F4000030FD
:1022A000F5000030F6008930F7008A150A12762012
:1022B0008A110A167008CC007108CD007208CE0091
:1022C0007308CF000A1200270A1670088316ED0063
:1022D0007108EE008030F00080306A067002031D45
:1022E00073296908003C0318CD2980306A06F00084
:1022F00080307002031D7E29093069020318CD2940
:102300006903F0000730F0054030700483120317B2
:10231000AB000A122E220A168316EB01EC010030E4
:102320006C02031D95295E306B020318C1298030B1
:102330006B0483120317AB000A122E220A168316AF
:102340006C086E02031DA6296B086D02031CB029E0
:102350003C3083120317B0000A121F210A16B62957
:1023600003178312B0010A121F210A160330FD0061
:10237000FD0BB829000000008316EB0A0319EC0AD4
:102380008F296903F0000730F00540307004831294
:102390000317AB000A122E220A1608008312031339
:1023A0000715071407110330FB008A30FC00553075
:1023B000FD00FD0BD929FC0BD929FB0BD929000005
:1023C0000000071521300317AB000A122E220A164F
:1023D00090300317AB000A122E220A16053003179D
:1023E000AB000A122E220A1613300317AB000A1292
:1023F0002E220A1620300317AB000A122E220A16CC
:102400002130FC007630FD00FD0B042AFC0B042A71
:1024100000000C300317AB000A122E220A160A1213
:10242000B7250A160230FB004530FC00A930FD003C
:10243000FD0B182AFC0B182AFB0B182A00000000C1
:10244000A501A6010A12A6220A1608008316031384
:1024500098169030831298008316871707138312FB
:102460008C1E352A1A08F0002F2A08008316031341
:102470008C120230E7000030E800EB01EC010A1298
:102480001E260A162A300317AB000A12C0210A16AC
:10249000700883160313E9007108EA0070088312BC
:1024A00003179E0071089F002430A0008A150A12AD
:1024B00030208A110A1624309E000A121C250A16A2
:1024C0000A121E260A162A08553A031D352B01301A
:1024D00083166902F0000030031C013E6A02F1001D
:1024E00070082A3E84000008233A031D352B8030F3
:1024F0006A06F00080307002031D802A14306902E1
:10250000031C352B1A30831203179E0017309F00CF
:102510008A150A1200208A110A1602308316031344
:10252000ED000030EE0080306E06F00080306A066C
:102530007002031D9D2A69086D020318CA2A6D08DE
:102540002A3E840000083B3A031DC62A6D082A3E35
:10255000840080016B08C03EEF0067082A3E8312AA
:1025600003179E000A125F270A16831603136F08CB
:102570008400700880006D08013EE70000300318F9
:10258000013E6E07E800EB0A0319EC0AED0A031995
:10259000EE0A932A01306902F0000030031C013E6C
:1025A0006A02F10070082A3E840080016B08C03E78
:1025B000EF0067082A3E831203179E000A125F2766
:1025C0000A16831603136F08840070088000400801
:1025D000831203179E000A127A260A167008031344
:1025E000D70083164108831203179E000A127A2629
:1025F0000A1670080313D6008316420883120317C5
:102600009E000A127A260A1670080313D200831657
:102610004308831203179E000A127A260A167008CE
:102620000313D80083164408831203179E000A126E
:102630007A260A1670080313D300831645088312FE
:1026400003179E000A127A260A1670080313D40094
:102650000A12A5240A168312AA018316EB01EC01C3
:102660008312D001D1018316E41283168C16080060
:10267000831603136708F000F00CF013F00CF0134E
:10268000F00CF013F00CF0130030F100A230F00762
:1026900017300318013EF1077008E2007108E300EB
:1026A0000A1218218A110A16F000680884007008BE
:1026B0008000680AF2000F306705F0000030F1007A
:1026C000A230F00717300318013EF1077008E2004E
:1026D0007108E3000A1218218A110A16F000720824
:1026E00084007008800002306807840080010800C0
:1026F0008B135530831203179E0054309F005330C4
:10270000A0005830A1005730A2005630A30052302C
:10271000A4008A150A12BD218A110A1683124A08DA
:1027200003179E0003134B0803179F00031356085B
:102730000317A0000A12EA250A168312CA0A03190F
:10274000CB0A4A0803179E0003134B0803179F0088
:10275000031357080317A0000A12EA250A1683126A
:10276000CA0A0319CB0A4A0803179E0003134B0831
:1027700003179F00031353080317A0000A12EA254A
:102780000A168312CA0A0319CB0A4A0803179E00C5
:1027900003134B0803179F00031354080317A000EB
:1027A0000A12EA250A168312CA0A0319CB0A4A0832
:1027B00003179E0003134B0803179F0003135508CC
:1027C0000317A0000A12EA250A168312CA0A03197F
:1027D000CB0A4A0803179E0003134B0803179F00F8
:1027E0000D30A0000A12EA250A168B170800831282
:1027F00003134B08F000F10103179E019F017008BD
:10280000A0000A12EA250A162130FC007630FD00ED
:10281000FD0B082CFC0B082C0000FF3083124A052E
:102820000317A00001309E0000309F000A12EA2525
:102830000A162130FC007630FD00FD0B1D2CFC0B30
:102840001D2C000008000034003400340034003433
:10285000003400345F340034003400340734003472
:102860000734003414347F3414347F341434243463
:102870002A347F342A341234233413340834643431
:1028800062343634493455342234503400340534FB
:1028900003340034003400341C3422344134003416
:1028A0000034413422341C340034143408343E34AF
:1028B00008341434083408343E34083408340034FE
:1028C00050343034003400340834083408340834C8
:1028D0000834003460346034003400342034103460
:1028E0000834043402343E345134493445343E34DF
:1028F000003442347F344034003442346134513443
:10290000493446342134413445344B34313418345D
:10291000143412347F34103427344534453445346C
:1029200039343C344A344934493430340134713414
:10293000093405340334363449344934493436349F
:1029400006344934493429341E340034363436349C
:102950000034003400345634363400340034083443
:102960001434223441340034143414341434143400
:102970001434003441342234143408340234013421
:1029800051340934063432344934793441343E34D4
:102990007E341134113411347E347F344934493457
:1029A000493436343E3441344134413422347F3466
:1029B0004134413422341C347F344934493449345D
:1029C00041347F3409340934093401343E3441340C
:1029D000493449347A347F340834083408347F3435
:1029E000003441347F3441340034203440344134A5
:1029F0003F3401347F3408341434223441347F347A
:102A000040344034403440347F3402340C34023497
:102A10007F347F340434083410347F343E344134FE
:102A2000413441343E347F340934093409340634A6
:102A30003E344134513421345E347F340934193406
:102A40002934463446344934493449343134013424
:102A500001347F34013401343F3440344034403455
:102A60003F341F342034403420341F343F3440344A
:102A7000383440343F346334143408341434633409
:102A8000073408347034083407346134513449341D
:102A90004534433400347F3441344134003402340B
:102AA00004340834103420340034413441347F3449
:102AB00000340434023401340234043440344034E9
:102AC000403440344034003401340234043400349F
:102AD000203454345434543478347F3448344434B7
:102AE000443438343834443444344434203438346E
:102AF0004434443448347F343834543454345434B3
:102B0000183408347E340934013402340C3452341D
:102B1000523452343E347F3408340434043478342C
:102B2000003444347D344034003420344034443460
:102B30003D3400347F3410342834443400340034BD
:102B400041347F34403400347C3404341834043449
:102B500078347C34083404340434783438344434DD
:102B60004434443438347C34143414341434083445
:102B700008341434143418347C347C340834043469
:102B80000434083448345434543454342034043431
:102B90003F344434403420343C34403440342034D6
:102BA0007C341C342034403420341C343C344034D5
:102BB000303440343C3444342834103428344434E1
:102BC0000C345034503450343C3444346434543431
:102BD0004C34443400340834363441340034003446
:102BE00000347F3400340034003441343634083447
:102BF000003410340834083410340834783446343F
:102C00004134463478344B3465347934623420347A
:102C1000433464346534733420343A3420340D340E
:102C20000A342D34203453345434413472347434DF
:102C300020347334613475347634653420342D3463
:102C40003E342034323434344C344334323435342A
:102C500036340D340A342D342034483441344C3465
:102C600074342034203473346134753476346534EC
:102C7000203478342034323434344C3443343234D5
:102C8000353436340D340A342D342034523445343E
:102C90004C346934743420343C342D3420342034A2
:102CA000663472346F346D342034323434344C34FE
:102CB00043343234353436340D340A342D34203430
:102CC000443455344D347034203461346C346C34B5
:102CD000203446346C3461347334683420346134C5
:102CE0007234653461340D340A3400344434693448
:102CF0006D3461346E3400344C3475346E34643465
:102D0000693400344D3461347234643469340034CD
:102D10004D34653472346334723400344A3465346B
:102D20007534643469340034563465346E34643434
:102D300072340034533461346D3465346434003497
:102D400000340034003400340034003450346C3427
:102D50006134743469346E34653420345034493409
:102D6000433431343634463420344E346F346B348B
:102D7000693461342034313437342D3430343334D1
:102D80002D3432343034313436340D340A34003496
:102D90000A340D34203449346E34693474342034A8
:102DA0004434533431343334303437342034703491
:102DB000613472342034643465346634613475347B
:102DC000743420340D340A34203400340D340A3481
:102DD00049346E3469347434203449346E34743474
:102DE000653472347234753470347434733420340E
:102DF000553441345234543420340D340A342034A0
:102E000000340A340D342034723465342D344C349B
:102E10006534633474347534723465342034443426
:102E20005334313433343034373420340D340A34AD
:102E3000203400340A340D344D346934733465342D
:102E40002034613420346C3427346834653475346C
:102E500072346534203452345434433420340D34C5
:102E60000A3400340D340A34523441345A34203494
:102E700049346434783420347334613476346534BE
:102E800045346534703472346F346D340D340A3423
:102E900000340D340A3453345434413452345434ED
:102EA0002034733461347634653445346534703499
:102EB00072346F346D340D340A3400345334543466
:102EC00041345234543420347334613476346534AC
:102ED00045346534703472346F346D3400344C349E
:102EE0006534633474347534723465342034453455
:102EF0004534703472346F346D342E3420340034E1
:102F0000533454344F345034203473346134763471
:102F10002F34453465346534703472346F346D3415
:102F20000034203449346E346434653478342034C9
:102F3000323434344C3443343534313432343D3427
:102F40002034003430343134323433343434353492
:102F500036343734383439344134423443344434E9
:102F6000453446344E34653478347434203449342E
:102F7000643478343D3420342034003420344134F7
:102F80004434433430343D3420340034203441342C
:102F90004434433431343D342034003454346934BF
:102FA0006D3465343A34203400344134443443348D
:102FB00031343D34203400344134443443343034EB
:102FC0003D3420340034FF3FFF3FFF3FFF3FFF3FD2
:102FD000FF3FFF3FFF3FFF3FFF3FFF3FFF3FFF3F01
:102FE000FF3FFF3FFF3FFF3FFF3FFF3FFF3FFF3FF1
:102FF000FF3FFF3FFF3FFF3FFF3FFF3FFF3FFF3FE1
:10300000831203138601FD30831686008614FF3079
:1030100083128500FF30831685008801FE308312FD
:103020008700C030831687008901FF308312890032
:1030300089148A110A12EF278A150A1664130330BD
:10304000FB008A30FC005530FD00FD0B2528FC0BF1
:103050002528FB0B25280000000083128910203052
:103060008316990018158A1126228A150230FB0052
:103070004530FC00A930FD00FD0B3C28FC0B3C2832
:10308000FB0B3C28000000000C300317AB008A113A
:103090000A12B4218A150A160330FB008A30FC009C
:1030A0005530FD00FD0B5228FC0B5228FB0B52281B
:1030B000000000008914A030EF00C930E700A630FE
:1030C00003179E0016309F000A1200200A168A116C
:1030D000CE218A15043083120313FB00CF30FC008D
:1030E0000130FD00FD0B7228FC0B7228FB0B7228CF
:1030F00000000000831664174030FB006A30FC00BB
:103100009730FD00FD0B8228FC0B8228FB0B8228E8
:10311000000000000A12EE270A160D30FB00AF3047
:10312000FC00B630FD00FD0B9328FC0B9328FB0B35
:1031300093280000861CA828C83003179E0016306C
:103140009F000A1200200A160A12DB270A16B1286D
:103150000130831203179E0017309F000A120020CF
:103160000A168316031364135530831203179E0047
:1031700054309F005330A0005830A1005730A200B7
:103180005630A3005230A4000A12BD210A16553051
:10319000E7005430E8005330E9005830EA00573077
:1031A000EB005630EC005230ED008A1100208A15F9
:1031B000831255088316E700831254088316E8002B
:1031C000831253088316E9000A12B8230A16580816
:1031D0008316E700831257088316E8008312560807
:1031E0008316E900831252088316EA000A124A2263
:1031F0000A161A30FB005E30FC006E30FD00FD0B3D
:10320000FF28FC0BFF28FB0BFF280000831664122D
:1032100064170430E7000030E8008A11CC208A15DA
:103220000317A5010430A6008A110A12A6228A15E6
:103230000A16831203136F0803179E00DC309F00E9
:103240001730A0008A110A1228268A150A160313BD
:103250006F080317A5008A110A12BD238A150A16E2
:10326000063083160313E7000030E8008A11CC20F3
:103270008A150317A5010630A6008A110A12A62294
:103280008A150A16831203136F0803179E00D530A0
:103290009F001730A0008A110A1228268A150A16E4
:1032A00003136F080317A5008A110A12BD238A159C
:1032B0000A168A110A121E268A150A1603300317E7
:1032C0009E0016309F000A1200200A16E630831274
:1032D00003179E0016309F000A1200200A168B0169
:1032E000831603138C1683121A08E6000B178B172C
:1032F000EB01EC018316E4108312E901EA01831665
:10330000E701E8010A1287270A1670088312E8000D
:103310007008E500E401E90A0319EA0A690883165E
:10332000E70083126A088316E8000A1287270A1644
:1033300070088312E8000030F10070086407CA00CA
:1033400065080318013E7107CB00913003179E00FA
:1033500017309F000A1200200A16A03083120313B0
:10336000EF004A0803179E0003134B0803179F0042
:1033700003136F080317A0000A1230200A16031364
:103380006F0803179E008A110A121C258A150A1657
:103390008A110A121E268A150A16DD01DE01DB01DA
:1033A000DC01AA01A030EF008312553003179E0004
:1033B00054309F005330A0005830A1005730A20075
:1033C0005630A3005230A4000A12BD210A1655300F
:1033D000E7005430E8005330E9005830EA00573035
:1033E000EB005630EC005230ED008A1100208A15B7
:1033F0006417831255088316E70083125408831656
:10340000E800831253088316E9000A12B8230A164B
:1034100083166413BE30831203179E0017309F007B
:103420000A1200200A16A03083120313EF0083163D
:10343000E7010A1258270A1670088312D90071088A
:10344000DA00700803179E0071089F0003136F08CD
:103450000317A0000A1230200A16831603136417FC
:10346000063083120317A5000430A6008A110A1241
:10347000A6228A150A16831203136F080317A500E4
:103480008A110A12BD238A150A169E019F01031391
:103490006F080317A0000A1235210A1664133B3087
:1034A00083120317AB008A110A12B4218A150A1677
:1034B00083166417831259088316E70083125A088B
:1034C0008316E8000530E9000030EA008A11372150
:1034D0008A150230831203138906A030EF00C6302C
:1034E00003179E0017309F000A1200200A16A03012
:1034F00083120313EF0001308316E7000A125827E6
:103500000A1670088312E2007108E30070080317BE
:103510009E0071089F0003136F080317A0000A1292
:1035200030200A168316031364170630831203171C
:10353000A5000630A6008A110A12A6228A150A16CC
:10354000831203136F080317A5008A110A12BD2303
:103550008A150A169E019F0103136F080317A00026
:103560000A1235210A16831262088316E7008312B5
:1035700063088316E8000730E9000030EA008A118A
:1035800037218A1583160313E418CB2A8A110A12ED
:103590001E268A150A1683166413E41E7B2D2A3014
:1035A000831203179E008A110A121C258A150A1617
:1035B0008A110A121E268A150A162A08553A031D70
:1035C0002D2B3D08233A031D2D2B8A1136228A15F7
:1035D0005530831203179E0054309F005330A000D3
:1035E0005830A1005730A2005630A3005230A4003A
:1035F0000A12BD210A165530E7005430E800533056
:10360000E9005830EA005730EB005630EC005230F9
:10361000ED008A1100208A15831255088316E700F1
:10362000831254088316E800831253088316E900B6
:103630000A12B8230A1658088316E700831257089F
:103640008316E800831256088316E9008312520895
:103650008316EA000A124A220A162A08523A031D61
:10366000502B2B08413A031D502B2C085A3A031DAE
:10367000502B00305C06031D3F2B03305B06031DFF
:10368000502B323003179E0017309F000A12002083
:103690000A1683120313CA01CB018A11F7238A1574
:1036A00083122A08533A031DA12B2B08543A031DF9
:1036B000A12B2C08413A031DA12B00305C06031DF1
:1036C000632B03305B06031DA12B493003179E00BB
:1036D00017309F000A1200200A168316031364177E
:1036E000C9308312E7000317A5010330A6008A1131
:1036F0000A12A6228A150A168312031367080317F3
:103700009E005E309F001730A0008A110A12282602
:103710008A150A16031367080317A5008A110A12EF
:10372000BD238A150A1683160313E4148312CA0AEA
:103730000319CB0A8A1178238A158312CA0A03193E
:10374000CB0A2A08483A031DF12B2B08413A031DE6
:10375000F12B2C084C3A031DF12B00305C06031DA5
:10376000B32B03305B06031DF12B83166417C9309E
:103770008312E7000317A5010330A6008A110A127D
:10378000A6228A150A1683120313670803179E00E0
:1037900080309F001730A0008A110A1228268A154F
:1037A0000A16031367080317A5008A110A12BD231E
:1037B0008A150A1601309E0000309F000313670827
:1037C0000317A0000A1235210A16E4108A11782383
:1037D0008A1506308312CA070318CB0A8A11F72309
:1037E0008A1583122A08523A031D732D2B08453A75
:1037F000031D732D2C084C3A031D732D00305C06FD
:10380000031D042C03305B06031D732D8316E41087
:103810006417C9308312E7000317A5010330A6001F
:103820008A110A12A6228A150A1683120313670840
:1038300003179E006F309F001730A0008A110A12F4
:1038400028268A150A16031367080317A5008A118C
:103850000A12BD238A150A16831603136413E7019F
:10386000E8010A1287270A1670088312E800700818
:10387000E500E40101308316E7000030E8000A1299
:1038800087270A1670088312E8000030F1006408E8
:10389000F00765080318013EF1077008CA007108B7
:1038A000CB00F00A0319F10A7008CA007108CB00B6
:1038B000C930E700700803179E0071089F000313CA
:1038C00067080317A0000A1230200A1603136708BE
:1038D00003179E008A110A121C258A150A168A11DE
:1038E0000A121E268A150A16C930E7000230E900BE
:1038F0000030EA0080306A06F00080307002031D5C
:10390000832C083069020318AA2C69088316E70083
:1039100083126A088316E8000A1287270A167008BD
:103920008312E80070088316E70083126708831685
:10393000E8008A1138238A158312670803179E004E
:103940008A110A121C258A150A160313E90A03199B
:10395000EA0A7A2C8A110A121E268A150A16C9301A
:10396000E7000830E9000030EA006A084B02031D56
:10397000BB2C69084A02031C732D06306902F30050
:103980000030031C013E6A02F4007308F000740862
:10399000F100F10CF00CF113711BF1177008E40049
:1039A0007108E5007008013E03179E0000300318FF
:1039B000013E71079F00031367080317A0000A1256
:1039C00030200A160313670803179E008A110A1293
:1039D0001C258A150A160930AB008A110A12B42177
:1039E0008A150A1669088316E70083126A08831687
:1039F000E8000A1287270A1670088312E800E90A0D
:103A00000319EA0A69088316E70083126A08831615
:103A1000E8000A1287270A167008F300F2018312E1
:103A200068087207F00073080318013EF10070087F
:103A3000E2007108E300700803179E0071089F0000
:103A4000031367080317A0000A1230200A16031395
:103A5000670803179E008A110A121C258A150A1688
:103A60000930AB008A110A12B4218A150A166208BD
:103A7000F0006308F1000A1240270A160030F40033
:103A80000030F5002030F6007730F7000A1256219A
:103A90000A167008CC007108CD007208CE007308B9
:103AA000CF0070088316E7007108E8007208E9008B
:103AB0007308EA00C930EB000330EC000A12FA2464
:103AC0000A16C930831203179E008A110A121C2598
:103AD0008A150A168A110A121E268A150A16E90A7A
:103AE0000319EA0AB52CAA018316E4128312DB013A
:103AF000DC01DD01DE018316E41C0B2E093083128C
:103B00000317AB008A110A12B4218A150A1683160C
:103B10006417C9308312E7000317A5010230A6001D
:103B20008A110A12A6228A150A168312031367083D
:103B300003179E00B2309F001730A0008A110A12AE
:103B400028268A150A1603134A0803179E00031332
:103B50004B0803179F000B30031367070317A000E0
:103B60000A1230200A16031367080317A5008A11EA
:103B70000A12BD238A150A1601309E0000309F00EC
:103B8000031367080317A0000A1235210A168312CF
:103B90006308F000F1017008E8004A0803179E006E
:103BA00003134B0803179F007008A0008A110A1224
:103BB000EA258A150A162130FC007630FD00FD0B3F
:103BC000DF2DFC0BDF2D00008312CA0A0319CB0A7C
:103BD000FF306205F0007008E8004A0803179E00F5
:103BE00003134B0803179F007008A0008A110A12E4
:103BF000EA258A150A162130FC007630FD00FD0BFF
:103C0000FF2DFC0BFF2D00008312CA0A0319CB0AFB
:103C10008A11F7238A15D4290C2EFF3FFF3FFF3F5F
:02400E00A62BDF
:020000040000FA
:1042000031003600460038003700370020007700C4
:10421000690074006800200042006F006F007400A5
:104220006C006F0061006400650072002000650092
:104230006E00200030007800310046003200380067
:1042400051003D00310030004D0048007A00200050
:10425000310039003200300030002000620064007C
:10426000730020000D000A000000FF00FF00FF00A7
:10427000FF00FF00FF00FF00FF00FF00FF00FF0046
:10428000FF00FF00FF00FF00FF00FF00FF00FF0036
:10429000FF00FF00FF00FF00FF00FF00FF00FF0026
:1042A000FF00FF00FF00FF00FF00FF00FF00FF0016
:1042B000FF00FF00FF00FF00FF00FF00FF00FF0006
:1042C000FF00FF00FF00FF00FF00FF00FF00FF00F6
:1042D000FF00FF00FF00FF00FF00FF00FF00FF00E6
:1042E000FF00FF00FF00FF00FF00FF00FF00FF00D6
:1042F000FF00FF00FF00FF00FF00FF00FF00FF00C6
:10430000FF00FF00FF00FF00FF00FF00FF00FF00B5
:10431000FF00FF00FF00FF00FF00FF00FF00FF00A5
:10432000FF00FF00FF00FF00FF00FF00FF00FF0095
:10433000FF00FF00FF00FF00FF00FF00FF00FF0085
:10434000FF00FF00FF00FF00FF00FF00FF00FF0075
:10435000FF00FF00FF00FF00FF00FF00FF00FF0065
:10436000FF00FF00FF00FF00FF00FF00FF00FF0055
:10437000FF00FF00FF00FF00FF00FF00FF00FF0045
:10438000FF00FF00FF00FF00FF00FF00FF00FF0035
:10439000FF00FF00FF00FF00FF00FF00FF00FF0025
:1043A000FF00FF00FF00FF00FF00FF00FF00FF0015
:1043B000FF00FF00FF00FF00FF00FF00FF00FF0005
:1043C000FF00FF00FF00FF00FF00FF00FF00FF00F5
:1043D000FF00FF00FF00FF00FF00FF00FF00FF00E5
:1043E000FF00FF00FF00FF00FF00FF00FF00FF00D5
:1043F000FF00FF00FF00FF00FF00FF00FF00FF00C5
:00000001FF
